:100000000C9438000C9466000C94ED000C94530092
:100010000C9453000C9453000C9453000C94530014
:100020000C9453000C9453000C9453000C94530004
:100030000C9453000C9453000C9453000C945500F2
:100040000C9453000C9453000C9453000C945300E4
:100050000C9453000C9453000C9453000C945300D4
:100060000C9453000C9453000C9453000C945300C4
:1000700011241FBECFEFD0E1DEBFCDBF12E0A0E064
:10008000B1E0ECE2FFE002C005900D92A038B107AC
:10009000D9F71FE0A0E8B2E001C01D92AE36B1076B
:1000A000E1F70C94FB030C9400001F920F920FB623
:1000B0000F9211248F93809180028F5F8093800232
:1000C0008F910F900FBE0F901F9018951F920F9257
:1000D0000FB60F9211248F939F93EF93FF93E091AC
:1000E0008102FF278091840090918500EE0FFF1F11
:1000F000E257FD4F91838083E0918102FF27809139
:100100008002E254FD4F8083E0918102FF27EA5292
:10011000F14F81E08083E0918102FF2780912901E6
:10012000F695FE2FEE27F795E795EA52FD4F858766
:10013000E0918102FF2780912A01F695FE2FEE279C
:10014000F795E795EA52FD4F8687E0918102FF27F8
:1001500080912B01F695FE2FEE27F795E795EA5251
:10016000FD4F8787E0918102FF2780912C01F69552
:10017000FE2FEE27F795E795EA52FD4F808BE09131
:100180008102FF2780912D01F695FE2FEE27F7952E
:10019000E795EA52FD4F818BE0918102FF27809124
:1001A0002E01F695FE2FEE27F795E795EA52FD4FC3
:1001B000828B809181028F5F809381028091810286
:1001C000883111F410928102FF91EF919F918F91EC
:1001D0000F900FBE0F901F9018951F920F920FB6A1
:1001E0000F9211242F933F934F935F936F937F93BD
:1001F0008F939F93AF93BF93EF93FF931DBA87EFB6
:1002000088B988B98FEF88B986B18171E9F3E09137
:100210008102FF278091840090918500EE0FFF1FDF
:10022000E257FD4F91838083E0918102FF27809107
:100230008002E254FD4F808386B18171E9F789EF36
:1002400088B988B988B988B940B193B18FEF88B9B6
:1002500020E030E077EF6FEF59EFEEEEFEE078B997
:1002600078B968B986B18171E9F3408391832E5FD3
:100270003F4F329686B18171E9F758B958B958B9EC
:1002800058B940B193B168B92E3F310541F7409359
:10029000EC0F9093ED0F80918D02833009F490C0A4
:1002A00080918D028823A9F59091EE0E97FDC6C02E
:1002B0008091EF0E87FDE1C0981708F0A2C040E0E2
:1002C00050E0AEEEBEE0E0918102FF27CA019695B4
:1002D00087952C911296F695FE2FEE27F795E795C8
:1002E000EA52FD4FE80FF91F20834E5F5F4F81E018
:1002F0004030580741F7E0918102FF27F695FE2F25
:10030000EE27F795E795EB5AFC4F80818E7F80832F
:100310002EC080918D02813009F492C041E050E0FE
:10032000AFEEBEE0E0918102FF27CA019695879566
:100330002C911296F695FE2FEE27F795E795EA5247
:10034000FD4FE80FF91F20834E5F5F4F81E0413082
:10035000580741F7E0918102FF27F695FE2FEE271F
:10036000F795E795EB5AFC4F808181608083E0919F
:100370008102FF27EA52F14F32E03083209181025F
:10038000809181028F5F8093810280918102883108
:10039000A9F19091810280918202981751F1809188
:1003A00083028F5F8093830280918302803120F4E7
:1003B0003CBB83E08DBB63C03CBB81E08DBB5FC0B9
:1003C00020E030E0AEEEBEE0E0918102FF278D91AB
:1003D000F695FE2FEE27F795E795EA52FD4FE20FCF
:1003E000F31F80832F5F3F4F81E02030380761F794
:1003F000BECF822F992780938102D1CF10928102A4
:10040000C8CF41E050E0AFEEBEE0E0918102FF27AF
:10041000CA01969587952C911296F695FE2FEE2798
:10042000F795E795EA52FD4FE80FF91F20834E5FDD
:100430005F4F81E04130580741F78CCF909538CF1E
:1004400040E050E0AEEEBEE0E0918102FF27CA013D
:10045000969587952C911296F695FE2FEE27F79597
:10046000E795EA52FD4FE80FF91F20834E5F5F4F7B
:1004700081E04030580741F73ECF80951DCFFF9176
:10048000EF91BF91AF919F918F917F916F915F910C
:100490004F913F912F910F900FBE0F901F90189585
:1004A0008F708A3018F0895C99270895805D9927AC
:1004B000089560E070E080917F028F7E80937F02DC
:1004C00020E030E040E050E080917F028BB92F5F68
:1004D0003F4F4F4F5F4F203888E3380781E0480790
:1004E00080E0580789F780917F02806180937F02C6
:1004F00020E030E040E050E080917F028BB92F5F38
:100500003F4F4F4F5F4F203888E3380781E048075F
:1005100080E0580789F780917F028F7D80937F026A
:1005200020E030E040E050E080917F028BB92F5F07
:100530003F4F4F4F5F4F203888E3380781E048072F
:1005400080E0580789F780917F02806280937F0264
:1005500020E030E040E050E080917F028BB92F5FD7
:100560003F4F4F4F5F4F203888E3380781E04807FF
:1005700080E0580789F780917F028F7B80937F020C
:1005800020E030E040E050E080917F028BB92F5FA7
:100590003F4F4F4F5F4F203888E3380781E04807CF
:1005A00080E0580789F780917F02806480937F0202
:1005B00020E030E040E050E080917F028BB92F5F77
:1005C0003F4F4F4F5F4F203888E3380781E048079F
:1005D00080E0580789F76F5F7F4F6430710509F03D
:1005E0006ACF0895982F80918502873028F5292FAA
:1005F000332780918502E0917302F0917402E80F35
:10060000F11D8081992787FD90952817390709F4F6
:1006100046C041E080918502E0917D02F0917E022A
:10062000E80FF11D8081992787FD909528173907DC
:1006300009F44BC0442341F5809185028F5F80937C
:10064000850280918502873080F01092850280912A
:100650008902873058F480918A02873038F51092E9
:100660008A0280918A0280938902089510928A02F8
:1006700080918A0280938902809184028F5F8093A7
:10068000840210928802089510928502809185025A
:1006900080938A0280918A028093890208958091D2
:1006A00089028F5F8093890240E0B4CF10928A0262
:1006B00080918A0280938902809184028F5F809367
:1006C000840281E080938802089580918A028F5F7E
:1006D00080938A02B1CF982F8C32A1F0809185024D
:1006E000841778F480918502262F280F312D311D33
:1006F000F901E45EFE4F9083809185028F5F8093C5
:1007000085020895809184028F5F80938402109205
:1007100085020895982F8C32F1F08091850284171C
:10072000C8F4903309F452C080918502462F480FD7
:10073000512D511DFA01E45EFE4F908381E08093BC
:100740008C029E3209F454C0809185028F5F8093A1
:10075000850208950895809184028F5F80938402BA
:1007600080918502841758F580918B02882381F44B
:1007700080918502262F280F312D311DF901E45E6D
:10078000FE4F8EE28083809185028F5F8093850289
:1007900080918502841798F4772790E380918502F1
:1007A000FB01E80FF11DE45EFE4F9083809185020E
:1007B0008F5F8093850280918502841778F3109271
:1007C000850210928B0210928C02089520918C0267
:1007D000213009F0B9CF80918502462F480F512D65
:1007E000511DFA01E45EFE4F908320938C02ACCF42
:1007F00080938B02A9CFCFEFD0E1DEBFCDBF11B880
:100800009FEF92B914B895B98EE087B998B980E78F
:100810008AB98FE88BB982E08093810081E0809370
:100820006F0015BE8BE08093690083E08DBB7894E8
:1008300086B1807282958695877080938D0289B18A
:1008400090918D0280788295869586958370892B0C
:1008500080938D0216B1107C80918D02833019F047
:100860008DE4809360010E945902103409F45BC347
:10087000103809F455C3112309F04FC390E08FE1FC
:100880009093C5008093C40088E18093C10086E006
:100890008093C200A0911A01B0911B018C91882312
:1008A00069F0FD0131968091C00085FFFCCF8C91ED
:1008B0008093C600DF0181918823A9F7FF248091EE
:1008C000C00087FD56C090918102809182029817E6
:1008D000B1F3E0918202FF27EA52F14F808181302B
:1008E00009F467C0E0918202FF27EA52F14F80814C
:1008F000823029F78091860290918702892B09F432
:10090000C0C18091860290918702019709F438C294
:100910008091860290918702029708F46FC18091BE
:100920008602909187028E50914008F067C18091B5
:10093000C00085FFC4CFE0918602F0918702E45A9F
:10094000FE4F80818093C600E0918602F09187027D
:10095000E45AFE4F8081F8268091860290918702AA
:10096000019690938702809386028091C00087FF52
:10097000AACF9091C60080918402882309F4D0C048
:1009800080918802882309F0B6C080918402853066
:1009900009F449C2863008F022C2823009F486C2C6
:1009A000833008F065C2813009F4ABC21092840232
:1009B0008ACF8091860290918702892B09F4B4C076
:1009C0008091860290918702892BD1F080918602D6
:1009D000909187020E97A0F48091C00085FF6FCFA1
:1009E000E0918602F0918702E55EFE4F8081809360
:1009F000C600E0918602F0918702E55EFE4FAACF25
:100A000080918602909187020E9770F18091860204
:100A100090918702449740F58091C00085FF4FCFA9
:100A2000809182029927E0918602F0918702969543
:100A3000982F882797958795E80FF91FEB52FD4F60
:100A400080818093C600809182029927E09186027E
:100A5000F09187029695982F882797958795E80FAC
:100A6000F91FEB52FD4F76CF80918602909187025D
:100A7000449740F0809186029091870282349105DC
:100A800008F4AACF80918602909187028234910562
:100A900009F461C1809186029091870283349105A7
:100AA00009F4C7C180918602909187028434910530
:100AB00009F4C5C180918602909187028534910521
:100AC00009F4CEC180917F02806480937F0280917F
:100AD0007F028BB910928702109286028091820267
:100AE0008F5F8093820280918202883109F403C271
:100AF00083E08DBBE4CE80918402853059F086304E
:100B000008F07FC1823031F0833008F0C3C18130FA
:100B100009F04CCF40E060E0892F0E946B03D3CEF8
:100B2000892F0E94F202CFCE80917F028F7B80932B
:100B30007F0280917F028BB9E0918202FF27E2540D
:100B4000FD4F808182958F700E945002809320011A
:100B5000E0918202FF27E254FD4F80810E94500203
:100B600080932101E0918202FF27EE0FFF1FE257E1
:100B7000FD4F80819181892F992782958F700E94E6
:100B8000500280932201E0918202FF27EE0FFF1FA7
:100B9000E257FD4F80819181892F99270E94500251
:100BA00080932301E0918202FF27EE0FFF1FE2579F
:100BB000FD4F80819181929582958F7089279F70DA
:100BC00089270E94500280932401E0918202FF272E
:100BD000EE0FFF1FE257FD4F808191810E9450026E
:100BE00080932501809186029091870201969093CF
:100BF0008702809386020EE0F02E61CE80918602FD
:100C0000909187028E50914009F4A5C08091860290
:100C1000909187028F50914009F40BC18091860218
:100C2000909187028051914009F409C18091860218
:100C3000909187028151914009F412C180917F0205
:100C4000806180937F0280917F028BB9109287022E
:100C500010928602809182028F5F8093820280913F
:100C60008202883109F44AC18091830281508093C5
:100C7000830280918302803108F021CE82E08CBB18
:100C800037CF80917F028F7E80937F0280917F0299
:100C90008BB9E0918202FF27E254FD4F808182955B
:100CA0008F700E94500280936201E0918202FF27C0
:100CB000E254FD4F80810E94500280936301E091D5
:100CC0008202FF27EE0FFF1FE257FD4F80819181C7
:100CD000892F992782958F700E945002809364011A
:100CE000E0918202FF27EE0FFF1FE257FD4F808148
:100CF0009181892F99270E94500280936501E0918C
:100D00008202FF27EE0FFF1FE257FD4F8081918186
:100D1000929582958F7089279F7089270E94500233
:100D200080936601E0918202FF27EE0FFF1FE257DA
:100D3000FD4F808191810E945002809367018091D4
:100D40008602909187020196909387028093860293
:100D50009EE0F92EB4CD8091C00085FFB0CD8F2DDF
:100D600082958F700E9450028093C6008091860207
:100D700090918702019690938702809386029FCD7F
:100D8000C0E0D0E009E611E0E0918202FF27F6958D
:100D9000FE2FEE27F795E795EA52FD4FEC0FFD1F6A
:100DA000808182958F700E945002F8018083E091CB
:100DB0008202FF27F695FE2FEE27F795E795EA5278
:100DC000FD4FEC0FFD1F808121960E945002F8011B
:100DD00081830E5F1F4FC038D105B1F6BDCD87307E
:100DE00009F498CE873008F44FC0883009F492CEC9
:100DF000893009F0DBCD46E064E1892F0E946B0366
:100E000062CD873009F468C0873008F483CE88301B
:100E100009F480CE893009F0C9CD45E064E3892F1B
:100E20000E948A0350CD4AE067E2892F0E946B033B
:100E30004ACD8091C00085FF42CD8F2D93CF809108
:100E4000C00085FF3CCD8DE08093C6008091860276
:100E500090918702019690938702809386022FCD0E
:100E60008091C00085FF2BCD8AE08093C60074CDB1
:100E7000833009F44CC0843009F098CD41E065E23C
:100E8000892F0E946B031FCD41E062E3892F0E94EE
:100E90006B0319CD833009F43DCE843009F086CD43
:100EA00040E060E0892F0E946B030DCD41E06BE0D4
:100EB000892F0E946B0380912701813499F08091E2
:100EC0002E0180FD0FC080917F02806280937F029F
:100ED00080917F028BB9F7CC42E06AE3892F0E94B0
:100EE0006B03F1CC80917F028F7D80937F02809194
:100EF0007F028BB9E8CC10928202FACD1092820266
:100F0000B3CE46E06DE0892F0E946B03DCCC49E054
:100F10006BE1892F0E946B03D6CC91E083E0B0CCCB
:0C0F200090E080E4ADCC90E081E8AACC29
:100F2C000D0A4669726D7761726520566572736938
:100F3C006F6E3A203237610D0A0000012442532CA7
:100F4C003030303030302C2D2C3030303030302CA4
:100F5C003030303030302C303030302E303030308B
:100F6C002C2D2C30303030302E303030302C2D2C8D
:100F7C0030303030302C30302C3237612A00244263
:100F8C00442C3030303030302C3030303030303049
:100F9C003030303030303030303030303030303045
:100FAC003030303030303030303030303030303035
:100FBC003030303030303030303030303030303025
:100FCC003030303030303030303030303030303015
:100FDC003030303030303030303030303030303005
:100FEC0030303030303030303030303030303030F5
:100FFC0030303030303030303030303030303030E5
:10100C0030303030303030303030303030303030D4
:10101C0030303030303030303030303030303030C4
:10102C0030303030303030303030303030303030B4
:10103C0030303030303030303030303030303030A4
:10104C003030303030303030303030303030303094
:10105C003030303030303030303030303030303084
:10106C003030303030303030303030303030303074
:10107C003030303030303030303030303030303064
:10108C003030303030303030302A00244750524D20
:10109C00432C006B022447504747412C007502FF3C
:00000001FF
